:10000000B00500200D220000092200000922000096
:1000100000000000000000000000000000000000E0
:1000200000000000000000000000000009220000A5
:10003000000000000000000009220000092200006A
:100040000922000009220000090300000922000023
:10005000000000007D06000000000000000000001D
:10006000CD0600001D10000009220000092200003A
:1000700009220000092200000922000009220000D4
:10008000000000000000000009220000092200001A
:1000900009220000092200000922000009220000B4
:1000A00009220000000000000922000009220000CF
:1000B00000000000092200000922000009220000BF
:1000C0000F4B104A984202D153695B0501E0536916
:1000D0005B045B0F09D1126803231340012B01D18C
:1000E00009480CE08020000209E0012B04D0022B1B
:1000F00004D1064B186802E0054800E00548704747
:100100000000014000020050001BB700000000206A
:100110001027000000805101F7B5061C0191171C43
:10012000FFF7CEFF0025041C430802209F4208D899
:10013000094A944201D91C1C0125201C391C02F0DB
:10014000FDF8019B011C2B4301353360694370604E
:10015000201C02F0F3F8FEBDFFFFFF00F0B585B0F4
:100160000393394B01911F68111C381C02F0E6F80B
:1001700005260290FF2501240298211C02F0DEF8DA
:1001800080235B04984213D8304A83181B0CDBB2DF
:100190001D1C022B00D20225EDB2291C02F0CEF864
:1001A00080235B02984203D8012808D086B207E07A
:1001B0006400013EE4B2002EDED1244E00E0061CB5
:1001C000211C6943381C714302F0B8F8013D013E1F
:1001D000071CEDB2B6B2012C08D0022C08D0042CBA
:1001E00008D0083C631E9C41023404E0042402E071
:1001F000002400E001240198154B42081968D20040
:10020000FF209040814395400D431D60019A59683D
:1002100095000720A840221C0C1CAA4084431443CC
:100220005C6099680822AA400A439A60039B701C8C
:100230005843642102F082F8054A0138AD1868621B
:10024000381CEE6005B0F0BD00000020FFFF00008C
:1002500000000440024BDA6D1143D9657047C04677
:1002600000000440F0B5174A85B00D1C6946041C17
:10027000C1CAC1C1126803200A60134A6B465169A2
:1002800000222263E060A260954218D08A01920F9A
:100290009200D65868083018291C02F04FF80B4B12
:1002A0000238984207D9E8003018291C02F046F8B5
:1002B0000009023802E0C0239B051843606205B0C4
:1002C000F0BDC0462826000000020050FFFF0000DD
:1002D000014B00225A607047FC000050054B5A68E1
:1002E000012A06D059225A6016225A6088225A6082
:1002F000F4E77047FC000050A023DB059A68012159
:100300000A439A6070470000F0B504260022C34BF0
:100310001E62C34B19681A60012900D87DE10227CB
:10032000C04A10681300384200D1B4E01068C0061B
:1003300017D50124BC4A1078A0431070072903D8B0
:1003400011780919C9B21170B8490878117841407B
:1003500011701278D20700D509E110211A688A437A
:1003600058E01068800679D5106830420CD14024DE
:100370001368334313601068A0431060072900D945
:100380004BE11368234306E180241068A04310600A
:10039000072902D8126822431A6040211A68186897
:1003A00052080A4001408A4200D036E104211A680E
:1003B0009F488A431A6019689C4A09062CD504781C
:1003C00015789C49E4B2EDB20D55047812789A4D37
:1003D000E4B2D2B22A55002214000578AA4204D809
:1003E0008D5C01326C40D2B2F7E7002C0FD10120B6
:1003F000924A1460924A1470924A01341070924AE0
:10040000FF341168214311601A6802431A601968A9
:100410008E4A0A401A6000E10178002905D13F2484
:100420001178A143802900D1A1E001781478814D91
:10043000C9B2E4B26C54017812787F4CC9B2D2B21E
:10044000625420211A688A431A6002780132D2B2BB
:1004500002700278102A00D989E0DEE07348027841
:100460005200D2B20270072903D802780132D2B208
:10047000027077490A780132D2B20A700A78072AE4
:1004800005D920201A6802431A6000220A70102140
:100490001A680A43BEE7802514686D022C406C4838
:1004A00063D04C1F022C04D811686A4B0B401360B8
:1004B000AFE01268D2060FD5674A1468640814606A
:1004C000082904D980241168A40221431160102155
:1004D0001A688A431A6012E0604A1468640814605B
:1004E000082904D980241168A40221431160102135
:1004F0001A680A431A6002780132D2B20270027896
:10050000122A34D80278122A00D086E08024524A77
:1005100052481168A402490811600168214202D1C1
:10052000116821431160046811686140116011680D
:100530004B4A914271D14B4A146801688C4211D1E7
:10054000002180203D4A400011601A6801310A43B1
:100550001A603C4A11703C490A6802430A601968F3
:10056000414A56E70168116001E0032915D81A686D
:10057000920704D501203D4A3D49127888541968F4
:100580003C4A0A401A600023314A1370284A13700B
:10059000324A1360304A13603FE0082939D9642990
:1005A00008D91A2113682B43136013688B43136017
:1005B000047032E00278122AD9D91A68324206D081
:1005C0001A683A431A601968224A0A401A600421DC
:1005D0001A680A431A601A6892071ED52349244CE8
:1005E0000A78632A03D900220A70227004E00132DB
:1005F000D2B20A700021A15408211A680A431A6075
:1006000019681D4A0A401A600023094A03701370D2
:1006100003E003780133DBB20370F0BDC04000504B
:1006200038010020C4010020B0010020000100209A
:100630003C0100207C000020010100207800002007
:1006400043010020A3030020A40300200FFFFEFFAE
:10065000A2030020FFFFFEFFAC01002044010020A8
:10066000FFFF03001401002001FFFEFF080000202F
:100670004801002000FFFEFFCBFFFEFF084B0949A9
:100680001A6A1A62084B1A6A1A62084B1A6A1A62C4
:10069000074A088850321378C3189BB20B80704702
:1006A000804000508C000020C040005000410050AD
:1006B00091000020044B4118884203D00278013099
:1006C0001A60F9E77047C046000005400122BD4BA3
:1006D00013B59A60BC4A136801331360BB4A1368B0
:1006E00001331360BA4A1378632B03D813780133AC
:1006F000DBB2137010780138102800D960E101F0E6
:1007000013FE11001D005F0125005F012A005F013B
:100710005F01700074005F015F015F015F015F01B5
:100720005F01ED00AB4B5B7F1B0704D5AA4B1B7829
:10073000002B00D044E16423137041E10F21A64B4C
:100740001B788B43702B00D03AE1F4E70F22A34BC8
:100750001A705A7034E18024A14B64011A689D49D3
:1007600001A8224219D01C689E4A22401A60CB7C04
:10077000002B0ED14B7F9B0607D59C2303704A7C30
:100780005D3B1340984AD35C24E0A32303700933F4
:1007900020E0A6230370503B1CE01A6822431A6035
:1007A000CC7C002C0AD14A7F3F23920601D58C7C59
:1007B00000E04C7880229200A21804E080239B0085
:1007C000E218C23BFF3B23409209874C92B2A25CE5
:1007D000E35C027043700B7F0221DB0700D4EFE083
:1007E000ECE00222814B1A70EAE0814A13689B0513
:1007F00035D580480378DBB2591CC9B20170022B91
:1008000003D911687C4B0B401360724BDB7E5A0797
:100810000FD50222754B79481A70037872499B09EB
:10082000CB5C6E4A13703F2300780340CB5C53705F
:10083000C6E01B0700D4C3E003226C4B6A491A7060
:100840006E4A13789B09CB18187F644B1870107888
:100850003F2202408A5C5A709A229A70B0E01020BF
:100860001368034200D1ABE0654C2378DBB2591C1E
:10087000C9B22170022B02D9136883431360614B04
:100880001A881B88FF2A02D8DBB2002402E0012468
:100890000133DBB24F4AD17E0222C8070BD5534940
:1008A00051480A709A09825C4C490A703F221340F1
:1008B000C35C4B7084E0114200D181E003214B4ABC
:1008C000117049499A098A18107F444A10703F20D4
:1008D0000340CB5C53700B5D937071E03D4A137F16
:1008E00011009B076CD5537F9B0629D5464B547C42
:1008F0001878844264D15878927C824260D19A7888
:100900003648E42A02D09A78EC2A11D1344A126887
:10091000520106D5DA783D498A5C92090270DB788B
:1009200024E0DA788A18527892090270DB7825E0A0
:100930009A78E72A02D09A78EF2A3CD1DB782FE028
:10094000254B5278187882423AD15A782348E42AC3
:1009500002D05A78EC2A1CD1214A1268520107D5DC
:100960009A782A498A5C920902709B78CA5C07E0EF
:100970009A788A185278920902709B78C9184A7836
:100980003F23134043700278174B9A5C0270427801
:100990000FE05A78E72A02D05A78EF2A0BD19B78D9
:1009A000772B08D1353303700D4B0F4A1B685B0161
:1009B000DB0FD35C43700D4B1978C9B2FFF77AFE99
:1009C00013BDC0460000014038010020D4020020C1
:1009D00043010020910000207C0000203D01002008
:1009E000C4010020FFEFFFFF382600001C0100209B
:1009F000A403002034010020FFFDFFFFA803002016
:100A0000E50000208E00002001010020C801002028
:100A10008021104B09011A68F0B50A431A600021C1
:100A20001A000D4D0D4E0E4F6B5C28009C46735CFA
:100A300034009C4502D013683B40136001311029FB
:100A4000F2D10023E25CD2B2C2540133102BF9D1AF
:100A5000F0BDC046C40100201D0100207C00002024
:100A6000FFF7FFFFFA2210B5134C0123920000217B
:100A70002000FFF773FB0123FA22190092002000E7
:100A8000FFF76CFBFA220123920002212000FFF7FE
:100A900065FB1222A368FF3213430022A360074BB9
:100AA0001A609C22920019689142FCD9A268044BFA
:100AB0001340A36010BDC04600000440D4020020D3
:100AC000EEFEFFFF764BF7B51A688023DB040700C4
:100AD0000D00134057D0734C235C8B4200D1DDE0F6
:100AE000FFF7FCFB01F0F6FB8023E5556E4C9B0005
:100AF0002068BE08C018B600801901F0F3FB03237C
:100B00001F409F402900FC33BB400200B9409A437C
:100B1000114308402700814207D1802320689B00B1
:100B2000C018801901F0F2FB28E08023206800241F
:100B30009B00C01801F0B8FB5C4DAE786B783606B0
:100B40001B04F6182B7838681B02F618584B04352E
:100B50001B5DF61880239B00C0180019310001F0BE
:100B6000D5FB802338689B00C0180019310001F0C4
:100B7000CDFB802304345B009C42DED101F07CFB82
:100B8000FFF7A6FB8AE00137FCB20320532C00D903
:100B900085E0082C03D1464A180013707FE0444BCF
:100BA0001B5D8B424BD0FFF799FB01F093FB3E4E50
:100BB000A7003068381801F095FBC3B23200FF2B54
:100BC00005D198432B1830680193381809E0FF2DA0
:100BD0000ED0284085420BD16B1E3068FF3B381881
:100BE0000193190001F092FB3068019938181EE05A
:100BF0002F4B10681D55002701F056FB2C4B2A4E39
:100C0000DB5D3068013BFF3B0193BB00C0180199DD
:100C100001F07CFB3068BB00C0180199013701F07E
:100C200075FB542FEAD130682249F930FF3001F0CA
:100C30006DFB01F021FBFFF74BFB1D4B1D55312CCC
:100C40000CD11B4B3334313318784121604301F010
:100C5000FFFBFA22231A920000211CE0322C0CD157
:100C6000134B3234323318784121604301F0F0FBEA
:100C7000FA22231A920001210DE0332C0ED10C4BE5
:100C80003134333318784121604301F0E1FBFA221B
:100C90000221231A92000848FFF760FA0120FEBDE6
:100CA000C4010020C8010020CC02002092000020D6
:100CB00091000020785634120000044010B5FFF770
:100CC0000DFB01F007FB044B0021186801F01EFB2F
:100CD000FFF712FB10BDC046CC020020802130B5CA
:100CE00080240748074B49000268224203D09D68D0
:100CF000054A2A4001E09A680A439A60F4E7C04630
:100D00001801002000000440FFFEFFFFB949BA4B64
:100D1000F0B50D681A680B68B84893430B60B84B80
:100D200002785C78944203D000229A7002785A705C
:100D30000E68B44CB44A0023F60606D523685B055A
:100D400001D5931C00E0D31CDB7F0E68F60702D5AB
:100D5000161DF67F33430E68B60702D5561DF67F83
:100D600033430E68760721D5961DF67F3343160070
:100D700035363678F60605D50126077833433743EE
:100D80000770DBB2160037363678F60604D5022730
:100D900006783B433E430670160036363678F60634
:100DA00004D5042706783B433E4306700E68360799
:100DB00021D5D61DF67F3343160035363678B60674
:100DC00005D501260778334337430770DBB2160099
:100DD00037363678B60604D5022706783B433E43BD
:100DE0000670160036363678B60604D5042706781F
:100DF0003B433E4306700868C00503D51000083029
:100E0000C07F03430868800503D5100028300078B0
:100E100003430868400503D51000293000780343D8
:100E20000868000503D510002A30007803430868DD
:100E3000C00403D510002B300078034308688004F9
:100E400003D510002C30007803430868400403D514
:100E500010002D30007803430868000403D510000B
:100E60002E30007803430868C00303D510004030DB
:100E7000007803430868800303D5100041300078F0
:100E800003430868400303D5100042300078034351
:100E90000868000303D51000433000780343086856
:100EA000C00203D510004430007803430868800274
:100EB00003D510004530007803430868400203D58D
:100EC00010004630007803430868000203D5100084
:100ED0004730007803430868C00103D5100048304C
:100EE000007803430868800103D51000493000787A
:100EF00003430868400103D510004A3000780343DB
:100F00000868000103D510004B30007803430868DF
:100F1000C00003D510004C300078034308688000FF
:100F200003D510004D30007803430868400003D516
:100F300010004E30007803430968002903DA1100DD
:100F40004F3109780B43D90710D58020216840051F
:100F500001420FD12C4938310E78FA2189007143B2
:100F60002A4E89B231802168014302E02068284975
:100F700001402160353212787F2A05D9234A128830
:100F8000002A01D1013293431D498A789A422DD01B
:100F90000124204A234206D018480078204202D07B
:100FA0009068204302E001249068A04390600220F2
:100FB000034207D0114C2478044203D010249068D7
:100FC000204302E010249068A04390600420034274
:100FD00008D00A4C2478044204D08024906864002D
:100FE000204302E094680C48204090608B70014BD5
:100FF0001D60F0BD30010020FC000020C802002070
:1010000008000020C401002091000020D002002030
:10101000FFFFFFEF00000440FFFEFFFFF7B50121D7
:101020007F4B804C9960804B1A68009352181A606D
:101030001A680A4200D1ABE0A3887C4A934202D8E6
:101040005B18A3800AE00022A179A2804B1CA37147
:10105000774B53331B788B4200D2A27120890A212F
:10106000013080B2208101F0EFF98FB2002F00D063
:101070008EE0704D704E2B783088DBB201939D234B
:101080005B005843642101F0E3F9019B6B4A80B295
:101090005B0098522B7810000133DBB22B702B7859
:1010A000642B00D92F700023642133802A78D2B2B8
:1010B0000132D2B2642A00D900225500455B0139C1
:1010C000C9B25B190029F3D1594DE3602A005232AD
:1010D0001278002A01D05343E360E120E368000165
:1010E00058432B005133197801F028F9544901F085
:1010F00025F9544B06001A88E0600193904235D0E0
:101100000023A7792381BA00A21810611A001800E1
:10111000E36053352978DDB2A94207D922009D004A
:101120001032AA58013380180122F4E7002A00D0B7
:10113000E060E06801F002F9013F019BBF0080B26E
:10114000E71918803B69002B03D1002E01D1019BC8
:101150001E80374B50331B78002B19D010213A4A90
:1011600013680B4313600022384B1A702289384BE6
:101170009A420DD900212E4B218150331B788B428E
:1011800006D01020304A1368034313602F4B1970A8
:10119000274D304E6B7F5B072CD52F4A11684B1CB7
:1011A0001360C823E87A4343994223D91368013B6B
:1011B00013601022294B1B681343284A1360284BE5
:1011C0001B68002B05D0236E264A934206D80533B0
:1011D00003E0236E002B01D0013B2366236E012B1D
:1011E00004D980223368D200134302E032681E4BD8
:1011F0001340336033689B033DD532681B4B520468
:1012000005D5009A11211268D20531D504E0009A63
:101210001121126852052BD59A688A432AE0C046EC
:10122000200001400800002018010020E703000012
:1012300091000020900000208C000020D8020020A7
:1012400040420F008E000020A4030020E500002093
:1012500087130000C4010020780000203001002026
:1012600068420050FF010000FFFBFFFF0000044048
:101270009A680A439A60924A1388002B03D0138815
:10128000013B9BB21380009B1B68DB0601D1FFF77B
:101290003DFD230064331A78511C1970697A91421C
:1012A00010D800221A7022006532137801331370AF
:1012B00022006632137801331370220067321378EC
:1012C00001331370230065331A78002A04D10120FA
:1012D0007C490B7883430B702B003A331B789A427E
:1012E00004D10127774801783943017029003D3145
:1012F0000978CB18934204DA0121724A13788B43A0
:101300001370230066331A78002A04D102206D4935
:101310000B7883430B702B003B331B789A4204D12C
:101320000227684801783943017029003E31097865
:10133000CB18934204DA0221624A13788B4313706C
:10134000230067331A78002A04D104205D490B7802
:1013500083430B702B003C331B789A4204D1042743
:10136000584801783943017029003F310978CB187A
:10137000934204DA0421534A13788B431370336881
:101380005B0519D52B0035331B789B0704D501214C
:101390004C4A13788B4313702B00022136331B7891
:1013A0000B4203D0474A13788B4313702B0037331B
:1013B0001B789B071ED518E02B00012135331B78C5
:1013C0000B4203D03F4A13788B4313702B00363304
:1013D0001B78DB0704D502213A4A13788B4313703C
:1013E0002B0037331B78DB0704D50421354A1378EB
:1013F0008B431370344B1B685B071DD52B003533B3
:101400001B78DB0604D501212E4A13780B43137099
:101410002B0036331B78DB0604D50221294A1378CA
:101420000B4313702B0037331B78DB0604D50421E4
:10143000244A13780B431370234B1B681B071CD5DE
:101440002B0035331B789B0604D501211D4A1378E8
:101450000B4313702B0036331B789B0604D50221F7
:10146000184A13780B43137037352B789B0604D535
:101470000421144A13780B43137022006832138836
:1014800001339BB21380FA22D200934217D9002273
:1014900013000E49885C002801D00133DBB2013211
:1014A000642AF7D180200A4A0A49137000220B6887
:1014B000800003430B60084B683422801A70F7BD2C
:1014C000D0020020C8020020300100204801002086
:1014D000A8030020A403002034010020F0B587B049
:1014E000FEF7FCFED84ED94BD94ADA491A60316072
:1014F0007321B160D849D94C0A6000228A609A6091
:1015000000F0E8FEC020800300F0ECFE0500D448A7
:1015100000F0E8FE0296A54211D000F0BDFEC0200A
:10152000800300F0C1FEC0202100800300F0EEFE29
:10153000F021CB48890100F0E9FE00F0A5FE00F0A3
:10154000DFFEC84E00253060306800F0CBFE336807
:10155000A800C01800F0C6FEC34C60550135542DDC
:10156000F5D12378A52B06D1237DAA2B03D0002308
:10157000BE4F01931EE0306800F096FE2378002BEA
:1015800004D12021BA4A13680B4313600025237D40
:10159000AA2B03D0B74B4033EB5C6355615D3368D6
:1015A000A8000139FF39C018013500F0AFFE542DF5
:1015B000EDD1DCE7802330689B00C018019BC01888
:1015C00000F090FE019BAC4DE854030A3B70030C05
:1015D0007B70019B000E043301931A008023B870C6
:1015E0005B0004379A42E5D13068F930FF3000F0F3
:1015F00079FEA24988420ED100F03EFE2021237FD1
:101600000B421DD080269E48F60402688B4332436D
:101610000260237714E03068F930FF3000F076FE86
:10162000012320211E009248964A07680F42E3D109
:101630005F1C1B0302D11368734013603B00F4E787
:10164000637821002B70E3793D31AB71237AEB7124
:10165000637C2B74A37C6B74237FEB76637F2B7787
:1016600023003A331B780A78D218FF2A01DDDB43C6
:101670000B70230021003B333E311B780A78D218CF
:10168000FF2A01DDDB430B70230021003C333F3197
:101690001B780A78D218FF2A01DDDB430B70220089
:1016A00051321378013B032B01D90123137022001F
:1016B0000F2304265332117863480B400133137013
:1016C000714A724B02219A60029B029A5B69704DCB
:1016D000334353616F4A00F0BFFD802180272E60A5
:1016E0006D4E6E4A09053000FEF716FD8022336804
:1016F000FF053B4333603368920513433360802317
:10170000FA228021664E5B002B60D2000905300072
:10171000FEF702FD8022336892051F43376033686D
:101720008021134333608023C2229B002B609200F0
:10173000AB585C4E090233400B43AB50802205216D
:101740005202414800F088FD2022029B02995B6909
:10175000A02713434B612821534BFF051960C12378
:101760002A609B00EA5819311640C0221202164323
:10177000EE50E0235B01BB6323006425313318780E
:101780004A4E684300F064FEFA222B1A92000021B0
:101790003000FEF7E3FC2300323318784121684320
:1017A00000F056FEFA222B1A920001213000333449
:1017B000FEF7D4FC20784121684300F049FEFA226C
:1017C0002B1A920002213000FEF7C8FCB368384A99
:1017D00007211343B3603000FEF73CFD3A6B354BF5
:1017E0003549134002223B633B6BFF3213433B639B
:1017F0003248FEF737FDFEF76BFD072280210827F0
:101800002F4B89011A701E4A13680B4313601C4842
:101810000122036804001342FAD003683B4200D05F
:10182000FDE0284A28491368DBB2CB18197D0E4B1E
:101830005C7801940468A40448D5502949D1006813
:1018400080034BD4597049E0C04000500040005024
:1018500055550000CFFF000080400050FEFF2FFFD5
:1018600004003000CC02002091000020C9010020BB
:10187000A403002038260000C80100207856341246
:10188000C4010020504200500C0031000002005002
:1018900000E100E00100010000000140A08601001D
:1018A00020000140FF00FFFF804100500000044085
:1018B00044040000FEFEFFFE90D00300000005403F
:1018C000C802002014010020B82600000068800330
:1018D00004D4587F800601D500F02EFC8020BB4C3C
:1018E00080022568054200D059705B788B4201D098
:1018F00000F022FC236803420AD11068B44B102484
:10190000C00502D51868204301E01868A04318609C
:1019100013689B0ADAB2272A08D0322A08D0362A5E
:101920000BD0372A0ED0CD2A12D003E00F2314E0BB
:10193000302312E0D82A0DD001E03C230DE0DC2A50
:101940000AD001E03F2308E0DD2A06D1FF2304E0AE
:10195000CF2302E0F02300E0FC239C4A10688003C0
:1019600028D41068800425D402242020234207D0E4
:101970003B4214D103421DD014689648204018E021
:101980003B4201D100F012FC034201D000F0FFFB0A
:1019900080241068E4002043106000F0F8FB8C4ABB
:1019A0008024034200D1EBE31068234200D1E5E339
:1019B00038431060854A884E1068800403D412684A
:1019C000039D920326D501251D405A0701D5022209
:1019D0001543DA0602D504221543EDB27B4C5B06B3
:1019E00002D53D43EDB211E0012D0FD1049B01332F
:1019F000DBB20493039B012B00D0A4E3049B802B58
:101A000008D9802223689202134323602268734B13
:101A1000134023606B461B79039573708CE3016858
:101A20006F4B0B4003606F4B19780568C9B26E4B62
:101A3000ED0500D400E10F261D78B543702D00D0D0
:101A4000FAE00168090500D4AFE21978C9438907B3
:101A50004DD1597877294AD101680C201D78890E1B
:101A600011402840082805D00C2829D0042800D08F
:101A700062E31FE01F249878A043E02800D05BE3D6
:101A800000201E000725B4782C40A04204DA520042
:101A90000130D2B2C0B2F6E79878C00600D54BE369
:101AA00098780A4003003B4002D0002A00D068E149
:101AB0001343A8E04C4B9B788B4200D03CE360E1A1
:101AC00045489978027F2023002902D0134319004A
:101AD00003E011001A43994302772568434B2268BB
:101AE0001B2013402360FEF7EDFF256049E13E4DCA
:101AF0002B789B0700D01FE36E782368F6B25B015A
:101B000029D50C232A7813400C2B24D1AB78002B39
:101B10000ED0AB78102B0BD0AB78112B08D0AB7854
:101B2000122B05D0AB781B2B02D0AB781C2B03D12A
:101B300022682E4B134023606878A978C0B2C9B2DE
:101B4000FEF7C0FF002801D1FFF7B8F88022236814
:101B5000D20413432360542E00D9EDE2802322687F
:101B6000DB041A4000D0E7E20C2329780B40082B55
:101B700005D00C2B54D0042B00D0DDE247E01F2110
:101B8000AB788B43E02B00D0D6E20720DF3B164931
:101B9000897801408A4204DA5B000132DBB2D2B2BA
:101BA000F5E7A9780C4AC90622D5A978394204D0AC
:101BB000697852185178194303E0697852185178BE
:101BC00099436878C0B2FEF77DFFDAE0C4010020D7
:101BD00030010020FFFBFFFF91000020FFDFFFFF2F
:101BE000FFFFFDFF3C0100207C000020FFFFFFFB0A
:101BF0006978521851780B40A978394002D0002BEF
:101C000000D0BEE00B43002B00D095E2B9E0AA78EB
:101C1000AB496B78CB185B78934200D08CE2B0E094
:101C20006878A978C0B2C9B2FEF74CFF002800D08E
:101C3000A7E0FFF743F8A4E01A78002A05D1802234
:101C4000236892001343236036E020689D4A0240D7
:101C500022609B4A507F80061DD51878557C8542AE
:101C600012D15B78907C98420ED102239648C25CD8
:101C70005D1ED2B201334255102BF8D1934A13782E
:101C8000013BDBB2137012E0D37C002B00D153E296
:101C90008D4A127808E018785578854207D0D27CB2
:101CA000002A00D148E21B789A4200D044E2864BD9
:101CB0005B78E42B00D13FE280221F20236892044E
:101CC000134323602268824B134023602268814BB8
:101CD000134023607C4B5A788243602A00D1ACE1E8
:101CE00007D8202A50D0402A00D1A6E1002A0ED0E1
:101CF00022E2A02A00D1CEE103D8802A00D157E108
:101D00001AE2C02A00D1FDE1E02A5AD014E20329E8
:101D100000D911E25A78D20611D5032259780A4027
:101D20009978022A00D08039654BC9B2DA7C8A42A0
:101D300000D101E21320D974FEF7C4FEFCE15A7809
:101D40000F231340012B08D0002B02D00F2B18D0EB
:101D5000F2E180222368520060E0594C637F0E2B31
:101D600004D00E211D206177FEF7ACFEE37C002B32
:101D700004D000211320E174FEF7A4FEFEF7BCFAA4
:101D8000DAE1FEF76FFED7E12268920500D5D3E1D4
:101D90004B4AD27C002A02D019788A420CD19A7818
:101DA00052B2002A04DA80212268C9000A4302E004
:101DB0002168494A0A4022609B785B0600D1BBE15A
:101DC00065E12268120500D4EFE05A78EC2A34D19C
:101DD0002268520125D59A78002A12D19A78102AC1
:101DE0000FD19A78112A0CD19A78122A09D19A78AF
:101DF0001B2A06D19A781C2A03D12168374A0A4047
:101E000022609878D978C0B2C9B2FEF75BFE00288C
:101E100001D1FEF753FF80222368D20413432360CD
:101E20008AE19878D978C0B2C9B2FEF74BFE002893
:101E300000D081E1FEF742FF7EE15A78EF2A00D020
:101E40007AE19A78772A19D11D48DD78017F573ACF
:101E5000224B002D05D0802011432268C00402438C
:101E600003E00A43027722681A402260256822684C
:101E70001B2013402360FEF725FE2560124A93784D
:101E80001E2B00D858E193782A2B00D954E1917881
:101E9000134BD07859181F390870012092781149D6
:101EA0001F3A90400A88024392B20A800E498A4241
:101EB00000D041E11A783E2A18D0FEF70FFFC04645
:101EC00091000020FFFDFFFF7C0000203C0100206E
:101ED000FFFEFFFFFFDFFFFFFFFBFFFFFFFFFFFB3B
:101EE000B101002074000020FF0F00005A78012A81
:101EF000E3D19A78002AE0D1DA78B22ADDD11A79D2
:101F0000012A14D15A79072A11D19A79002A0ED1BF
:101F1000DA79002A0BD11A7A282A08D15A7A052AA6
:101F200005D19A7A202A02D1DB7A182BC5D0FEF788
:101F3000D5F900F0CFF9A34C0025206800F0B4F9E2
:101F4000A14B20685E5DAF00013EFF3EC01931002D
:101F500000F0DCF920683100C019013500F0D6F935
:101F6000402DEDD120689949FD30FF3000F0CEF9C9
:101F700000F092F9C020800300F096F9C020944947
:101F8000800300F0C3F9F0219248890100F0BEF906
:101F900000F07AF90321904A13680B43136000F0B4
:101FA0006BF98E4A8E4B1A60FEE7FEF731FDC3E0F7
:101FB000042900D9C0E084498A4A4D7FCC7CAD0712
:101FC00020D51D78AC4205D10F204C7D010015684D
:101FD000A14321E0002C0BD0487D0F215C78084004
:101FE000210081435970010014682039214001E02B
:101FF00011688143116058781F23116803400B4317
:10200000136099E01D780F20AC420DD14C7D15680E
:1020100021000140C943C9B21039294011605978E3
:1020200013680C40204005E0116881431160597825
:1020300013680840184310607EE004297CD8624889
:10204000427F92070BD410255978664A294203D063
:1020500011680D43156002E01168A9431160226800
:10206000920569D4C27C002A02D019788A420BD129
:102070005A78920604D580212268C9000A4302E0FA
:102080002168594A0A4022605B78DB0654D000225E
:10209000564B1A8050E004294ED859784A4AC9064E
:1020A00020D51C78D57C4F495148A54211D1547D8B
:1020B0000F222240D243D2B20D68120202431540D1
:1020C0000D605A7824090B6814402402E4180C604F
:1020D00032E00A6810400F2208605B7808681340FD
:1020E0001B020DE01978D27C8A4225D03D49414A35
:1020F000086802400A600F225B78086813401B03DF
:102100001B1818E030491A78C97C914214D05A78CB
:102110003449DE2A07D10868374A02400A609B78B2
:102120000A681B0406E00A681202120A0A609B7819
:102130000A681B0613430B60304A314B11680B4091
:102140001360FFF764FB23689B0300D456E48022EE
:102150002368D20113420CD06B461B797370059B28
:10216000581EC0B2FEF7AEFC2268264B1340236017
:1021700044E423680591134323603FE4B84318E423
:102180001068234201D0012409E001240BE09A06E3
:1021900000D40FE40424134A180603D51068204322
:1021A000FFF707FC1068A043FFF703FC034201D1CF
:1021B000FFF700FC0B4A1806F4D5106804431460BE
:1021C000FFF7F8FBCC02002091000020A5AA55A53E
:1021D0007EFFAFFF0400300000C000500400FA058D
:1021E0000CED00E030010020FFFBFFFF7400002039
:1021F000FFF0FFFFFF0FFFFFFFFF00FFC401002004
:10220000FCFFFEFFFFBFFFFFFEE7000008B5002355
:102210000C4A0D499A188A4204D20C49C95C013310
:102220001170F5E70A4B0B4A591C013B934203D24C
:1022300000221A700B1CF6E700F01CF8FFF74EF9AD
:1022400008BDC0460000002008000020EC27000068
:1022500009000020AC03002010B5130E84698B40E8
:10226000234312028361120AC3698A40111C194375
:10227000C16110BD70470000024B01211A688A43FA
:102280001A60704700C00050024B10211A688A4340
:102290001A60704700C00050024B10211A680A43B0
:1022A0001A60704700C00050094B2222DA600122F8
:1022B00058601A6118690121054A0840FAD111686D
:1022C0004023194202D00120136040427047C046AB
:1022D00000C00050024B01211A680A431A6070477F
:1022E00000C00050054B0022DA60012258601A61DC
:1022F0001A69D107FCD4014B9868704700C00050A0
:10230000014B58697047C04600C00050054B212260
:10231000DA600122586099601A611A69D107FCD409
:102320007047C04600C0005003B4714649084000E1
:102330004900095A49008E4403BC704700224308F3
:102340008B4274D303098B425FD3030A8B4244D37D
:10235000030B8B4228D3030C8B420DD3FF220902BF
:1023600012BA030C8B4202D31212090265D0030B7E
:102370008B4219D300E0090AC30B8B4201D3CB0374
:10238000C01A5241830B8B4201D38B03C01A5241B6
:10239000430B8B4201D34B03C01A5241030B8B42B8
:1023A00001D30B03C01A5241C30A8B4201D3CB02A3
:1023B000C01A5241830A8B4201D38B02C01A524188
:1023C000430A8B4201D34B02C01A5241030A8B428B
:1023D00001D30B02C01A5241CDD2C3098B4201D3A3
:1023E000CB01C01A524183098B4201D38B01C01A21
:1023F000524143098B4201D34B01C01A5241030998
:102400008B4201D30B01C01A5241C3088B4201D346
:10241000CB00C01A524183088B4201D38B00C01AF3
:10242000524143088B4201D34B00C01A5241411A1A
:1024300000D20146524110467047FFE701B5002027
:1024400000F0F0F802BDC0460029F7D076E77047EB
:1024500003460B437FD4002243088B4274D3030905
:102460008B425FD3030A8B4244D3030B8B4228D3A6
:10247000030C8B420DD3FF22090212BA030C8B42CC
:1024800002D31212090265D0030B8B4219D300E06C
:10249000090AC30B8B4201D3CB03C01A5241830BF1
:1024A0008B4201D38B03C01A5241430B8B4201D3A1
:1024B0004B03C01A5241030B8B4201D30B03C01ACA
:1024C0005241C30A8B4201D3CB02C01A5241830A44
:1024D0008B4201D38B02C01A5241430A8B4201D373
:1024E0004B02C01A5241030A8B4201D30B02C01A9D
:1024F0005241CDD2C3098B4201D3CB01C01A524104
:1025000083098B4201D38B01C01A524143098B428C
:1025100001D34B01C01A524103098B4201D30B0175
:10252000C01A5241C3088B4201D3CB00C01A52419A
:1025300083088B4201D38B00C01A524143088B425F
:1025400001D34B00C01A5241411A00D201465241F8
:10255000104670475DE0CA0F00D04942031000D317
:102560004042534000229C4603098B422DD3030A6C
:102570008B4212D3FC22890112BA030A8B420CD37C
:10258000890192118B4208D3890192118B4204D3A5
:1025900089013AD0921100E08909C3098B4201D325
:1025A000CB01C01A524183098B4201D38B01C01A5F
:1025B000524143098B4201D34B01C01A52410309D6
:1025C0008B4201D30B01C01A5241C3088B4201D385
:1025D000CB00C01A524183088B4201D38B00C01A32
:1025E0005241D9D243088B4201D34B00C01A524109
:1025F000411A00D20146634652415B10104601D396
:102600004042002B00D54942704763465B1000D31F
:10261000404201B5002000F005F802BD0029F8D0C5
:1026200016E770477047C046001BB7000000000067
:102630000080510100805101ACAAA9A5A3A69C9AD3
:10264000999593968E8D8BB1B2B4B874726C6A6999
:102650006563665C5A595553564E4D4B4771E8E4D5
:10266000E2D1C9C5D8D4D2CAC6CC78171B1D1E2E3C
:10267000363A272B2D353933A503FFFFFFFFFF1116
:102680003E00FF0AFFFFFFFFFFC0FF00FF00FFFF4C
:10269000FFFFFF00030EFFFFFF0204010000000028
:1026A000000000000000000000404040000000006A
:1026B0002000000000FFFFFF0000000000000000FD
:1026C00000000000000000000B01570450025101FF
:1026D0000608520791B1BFA1030554041214551303
:1026E000181A561992B257A215175816C1C959C5CA
:1026F000D9E15ADD93B35BA3CDD55CD1090B5D0A5B
:102700000F115E1094B45FA40C0E600D3638613763
:102710003C3E623D95B563A5393B643A484A6549FC
:102720004E00664F96B667A64B4D684CC2CA69C646
:10273000DAE26ADE97B76BA7CED66CD23F416D4026
:1027400045476E4698B86FA842447043E5E771E686
:10275000EBED72EC99B973A9E8EA74E9F7F975F849
:10276000FDFF76FE9ABA77AAFAFC78FBC3CB79C74D
:10277000DBE37ADF9BBBC0ABCFD77CD3EEF07DEF42
:10278000F4F67EF59CBC7FACF1F380F21B1D811C3E
:10279000212382229DBD83AD1E20841F2D2F852ED7
:1027A000333586349EBE87AE30328831C4CC89C87A
:1027B000DCE48AE09F538BAFD0D88CD424268D25BF
:1027C0002A2C8E2BA07B8FB0272990285F736963FA
:1027D0006865725F3E0100B20107000028052018FD
:0C27E000000000002F7369636865725FE1
:0827EC000080510116000000FD
:00000001FF
